:100000009FC7B9C7B8C7B7C7B6C7B5C7B4C7B3C71F
:10001000B2C7B1C7B0C74FCAAEC7ADC7ACC7ABC791
:10002000AAC7A9C7A8C7A7C7A6C7A5C7A4C7A3C764
:10003000A2C7A1C7A0C79FC79EC79DC761756775A7
:10004000757567757575757563757567757575758E
:100050006175756763636163756167756375637502
:1000600061677563616775677567757561617563EC
:100070007575616361616363616761616375636124
:1000800061757561636363636375676361756163FC
:1000900061637561617575637575756361636163CE
:1000A0006775676775677575756175756163636396
:1000B00075676163616161677575757563616761B6
:1000C0007563637563616775757575616361757572
:1000D0006361616375636167676163757567757592
:1000E0006375756163637575756375757575636340
:1000F000616175677575616375756767757563634C
:100100006175676375617561636175677563756353
:10011000756767676163636161756767756163755B
:100120006161676167677575756761756161636353
:100130006375677563637561636361757575616127
:1001400075676175676775677575756175757575BF
:10015000676375756363616375676167616167751F
:10016000637561616361756161756161676167672D
:1001700063756767617575757575676775616375B3
:1001800061637575756167617575636761616761E5
:1001900063636361677563636375616375756175D7
:1001A00075677575616175616163676375616375B5
:1001B0006161756775756775756175756161616791
:1001C000756375677567616175757563616175756F
:1001D000757567756161756761756363617575755F
:1001E0007575676767756775757561757561636343
:1001F00061636161616161636161636161616167E3
:100200007575676761756767616161677567616764
:10021000757563616761677575756175756375611E
:100220006775676367616175616175756763616350
:1002300075757575676161756175677563756375EA
:1002400063616763637575757563757561756767F8
:10025000616363757567616167676161616163614E
:100260006767677561617575756361616161617506
:1002700063757561676767616175757567756775C2
:1002800075756161676161756175756761756767CE
:10029000757561757575756161616175617561759A
:1002A00075637561616763616361636763637561EA
:1002B0007575616175757561677567636775676188
:1002C0007563756363637563616767677575757576
:1002D0007563676763757575616761616363617590
:1002E000756767756167617575756763636161756A
:1002F0006167677561757561616361756361637578
:100300006167677575756361616163757575616353
:10031000757567637575756163617561676161673F
:100320007575617575756761637563637567677505
:1003300067617575637575637575636167677575F5
:10034000676761636167637567677567637567632F
:1003500061676375756175756175677567676775E1
:100360007561756375756361616363756167676105
:1003700063757575756375617575616161617561C9
:10038000756161756761616161756767616163630B
:1003900061757561636167617567637567756167CD
:1003A00061637567756763616375756761636363CF
:1003B00075637563756361676161616361616167DD
:1003C000756775616367757567616161756363758D
:1003D00075636163756775616761616161616767B5
:1003E000616175637561756361616163757563757D
:1003F0006161637575756167616775636361616389
:100400006361616361676161756375617575677566
:100410007561676175757563637561617561757522
:100420006163616161637575677567636363757542
:1004300075756767756761616775757575756161F4
:100440006367636361636361676175757567636142
:1004500075637567757575617567637575676761D0
:100460006163616767616167616761617563616746
:1004700063616163756775677575676375676175D6
:1004800075617575637567756363756175617561B0
:1004900061757563636763617563617575757563B0
:1004A000636163757575756161677567757561758C
:1004B00067676167756775637563637561637561A8
:1004C0006161757561616175676175637563756794
:1004D0006375757561637561617567756375617560
:1004E000676361676175756361757575677561616E
:1004F0007575616761676775676175676161677564
:10050000636167616361616175636763756363619B
:10051000676767636161616375676761616167618F
:10052000757567637567617575617561617575610D
:100530007561616175756163636167617567617537
:100540007575756163616767637567636775756105
:1005500075616763757567676161757563756161FD
:1005600063616175637575676175756375616167F1
:1005700067757567677567677561617575617561C1
:1005800061757561636375677561756167617575BF
:1005900067757575616767616167756375616175B9
:1005A00063756361616163637575757567616761C3
:1005B00067616761756175757563616163756761B1
:1005C00061617563756175636167676363676775AB
:1005D00061676361636163637575677561617567A1
:1005E0006775677575676161676775757575616151
:1005F0007575677575616375757563637575756117
:10060000636161756361756175676775757563634E
:100610006161636363616375616175676775677560
:100620007567677575616363616163636175616354
:100630006167616775616775616775616375757518
:100640006375757575676161637575637561636100
:10065000756763616363616763616163756775751E
:10066000756775676761636375616161616167750E
:1006700063756163756161757575676775756161CE
:1006800061616163616161756775677563616175FA
:1006900075756361616375756361617567677575AC
:1006A00075616163616767636163616767756775DA
:1006B000756375756163756761677563756161639E
:1006C0006161616161677575756375676363757590
:1006D00075636361616361617575756767636167A0
:1006E0006167616361757567637567616361637590
:1006F0006163756761756763756775636367756760
:100700006175636361636167616361637575676187
:10071000676175756375756761636175756163613F
:1007200063636175677575637575757567677567FB
:100730006775677563616775677575617561616315
:10074000616363616767616163616161756163755D
:100750007563756161636361676775756763756705
:1007600075756375757561756361676761756775C3
:100770007561616375676361636167616167756313
:1007800063637567757567637561757563617567B3
:1007900063616761756361616375756163756363E7
:1007A000756163757567676367756775757561757D
:1007B0007563756163616767757563756161756799
:1007C000757575757563616161636163677567638D
:1007D000616767637567757575616175616767677F
:1007E00067637567616163617567756361616361A3
:1007F0006163756361756175676167756775676169
:10080000636175616363636175756767756763616C
:10081000676775617561756763676375616775752E
:100820006175636167616375636167616375616168
:10083000757563756363756367676367676763612E
:100840006367756167756775616763756167756310
:100850006161756363617563617575676363756114
:1008600063616375617567756361637575676775E6
:1008700067636167616161617575636167757567FC
:1008800063757561637563756161756161637563D6
:1008900075617575676363617561636363616361E6
:1008A000616175757575616375617575616775678A
:1008B00075756163636163616761616175756375B6
:1008C00061636361677567756375617567616363AC
:1008D00061616761636175636167756167617575A2
:1008E000677561636161756775616361757575676A
:1008F0007567677567617575636161637567616168
:100900007567636167636161756375757575677533
:100910007567636161756175676763616775757533
:100920007575677561636163616175756161616347
:100930006367756763757575616163756767616125
:10094000756167637567757567616163616167612B
:100950006361616161616361636363616167616177
:1009600067757575757567636163616167756361E7
:100970006161636161617575756163616161616325
:10098000616363616363616175756161616761750D
:100990007575756767756767757575756161757567
:1009A00075757563616361616175617575616363B7
:1009B00061676175636361756361616161636361EF
:1009C00061676361616761676775636175757561AB
:1009D0007575676161676175637561637575757557
:1009E00063616163616161677567616361637575A7
:1009F0006763616761756763756767637575636171
:100A00007563616161636161756175676775676170
:100A1000757567636375756767756761756175750A
:100A20006763756763756167616761636375636158
:100A30007575756775676361636161616167757518
:100A40007561616367676363757561637567757504
:100A500075756763636163637575756763756361F6
:100A6000636167617567616161756761757567630A
:100A700075636161756163616375756375676361F2
:100A800063756775756167636767677561636161E2
:100A900075636163757563756767757567676163AE
:100AA0006375757567677567636167677567637594
:100AB00067636175756163616161756163636175C8
:100AC0007575676375617567636161617567676394
:100AD000757561756167677575756161756767754E
:100AE000617575676761677575616361636167618A
:100AF0006175677575637563756175676167616158
:100B00006363616161616175756761757567636371
:100B10006161636361617575756161756167756751
:100B2000637561757567676361616161757563613F
:100B3000616761637563616375757563757563631B
:100B40006163616763616167756763616375756739
:100B5000676161616163757563616167617567751F
:100B60006767756361616363616161617567636133
:100B70006361616763757575616161636163676313
:100B800075756775756161616361616375756167CD
:100B900063756363616175757575676775676361B3
:100BA0006175757563616167756775757575616187
:100BB0006175676175617563637575756361636799
:100BC0007563757567616361616167757567616795
:100BD0006763756761616775676361616175756793
:100BE0006175616767757567617563616361676783
:100BF0006361676163757563616161677575756769
:100C0000636167616361756175677567616375636A
:100C10006161636161757561617575616761676364
:100C2000756763616761616175636167616763755A
:100C300075637567637561617563757567637567FE
:100C40006375616375616161617567756361676132
:100C500067756775677561637575676761636161FE
:100C600075636161616161676167757567617575FC
:100C700075757567756767616161676767637561DA
:100C800075636175637575617567756363757563A4
:100C900063637563616775636167636163637563EC
:100CA0006175676775677561677563757563757578
:100CB000676361756775676163757561756775638E
:100CC00063637567636163616167616161616761E6
:100CD00061637575636163616163756763756363A0
:100CE0007567636361757575677563617567617550
:100CF000676761616161676361636163757575638E
:100D00006375636775676161676775677563757537
:100D10007567757575636161617567676361636147
:100D20006361637567677575756775616163616335
:100D30006161616767616175757575756175676119
:100D40006163636163616161756361757561637539
:100D50006163616761636161636163617575756733
:100D600075677563756767756161637567756761D9
:100D700075677575677561617561676761617575BF
:100D800067756361616361616361636167757575EF
:100D900061756761756363757575676361616363C9
:100DA00075676161757561676163756361757563A9
:100DB00061616767616767616775756167617561C3
:100DC0006161756175757575616167616175636193
:100DD000756163617563616363616761756775758B
:100DE000676175757561676775676163617563755F
:100DF0006375676763617575616175676375756351
:100E0000616775756775616161636175756361615E
:100E10006161616761616175756761636367636380
:100E20007563616175676167677575676363616144
:100E3000676161757575616161756761617563751C
:100E4000637563617563676175637563636161672A
:100E50006161637575676761616167756175676118
:100E60006763616775617561756161616175676708
:100E700063636175676775616361757575676763DE
:100E800075616767757575756175616763756767A6
:100E900063757567617575676363617561677561B2
:100EA00061756767756761636161757561756763B2
:100EB000757575676375677561756761636361678C
:100EC0007575676375677561677575677563756354
:100ED0006161676767637567757567757563757554
:100EE000677567676175636375676375676361617C
:100EF0006175757567617567616167616367616376
:100F0000756375676167636361677567637563615F
:100F1000616167676167756361616175756163616F
:100F20007575616361636175616161636761616367
:100F300075754E000102048040201008040201086B
:100F400011241FBECFEFD2E0DEBFCDBF21E0A4E071
:100F5000B1E001C01D92A131B207E1F711E0A0E0BC
:100F6000B1E0EEE1FAE102C005900D92A430B107C4
:100F7000D9F758D452C544C8E8D2DC01CB01885710
:100F80009C4EAF4FBF4F8093040190930501A093F7
:100F90000601B0930701089560E08AE05ED360E047
:100FA00089E05BD360E088E058D360E087E055D308
:100FB00060E083E052C3F0DF61E08AE04ED360E09E
:100FC0008AE099D361E089E048D361E089E093C386
:100FD000E3DF61E08AE041D361E08AE08CD361E045
:100FE00089E03BD360E089E086C3D6DF61E089E039
:100FF00034D360E089E07FD361E088E02ED361E004
:1010000088E079C3C9DF61E089E027D361E089E046
:1010100072D361E088E021D360E088E06CC3BCDF7C
:1010200061E088E01AD360E088E065D361E087E0A2
:1010300014D361E087E05FC3AFDF61E088E00DD3E8
:1010400061E088E058D361E087E007D360E087E0A3
:1010500052C3A2DF61E087E000D360E087E04BD3BA
:1010600061E083E0FAD261E083E045C395DF61E0AF
:1010700087E0F3D261E087E03ED361E083E0EDD228
:1010800060E083E038C388DF61E08AE0E6D260E0B8
:101090008AE031D361E088E0E0D261E088E02BC3F0
:1010A0007BDF61E08AE0D9D261E08AE024D361E0AD
:1010B00088E0D3D260E088E01EC36EDF61E089E0A3
:1010C000CCD260E089E017D361E087E0C6D261E06E
:1010D00087E011C361DF61E089E0BFD261E089E0B0
:1010E0000AD361E087E0B9D260E087E004C3CF9320
:1010F000DF93CCE3D0E08FE0C333D80709F44DC0D1
:10110000FE018491813671F456DF61E070E080E089
:1011100090E04ED284DF61E070E080E090E048D261
:10112000B2DF2FC0853771F453DF61E070E080E0FB
:1011300090E03ED281DF61E070E080E090E038D264
:10114000AFDF1FC0873671F450DF61E070E080E0F0
:1011500090E02ED27EDF61E070E080E090E028D267
:10116000ACDF0FC0833691F44DDF61E070E080E0CA
:1011700090E01ED27BDF61E070E080E090E018D26A
:10118000A9DF61E070E080E090E012D261E070E001
:1011900080E090E00DD22196AECFDF91CF910895FF
:1011A000CF92DF92EF92FF92C12CD12C760103DF18
:1011B000C701B601FDD10CDFC701B601F9D115DFBA
:1011C000C701B601F5D11EDFC701B601F1D127DF96
:1011D000C701B601EDD130DFC701B601E9D139DF72
:1011E000C701B601E5D142DFC701B601E1D14BDF4E
:1011F000C701B601DDD154DFC701B601D9D15DDF2A
:10120000C701B601D5D166DFC701B601D1D18FE0E4
:10121000C80ED11CE11CF11C8BE4C816D104E104FA
:10122000F10429F6FF90EF90DF90CF900895CF92D0
:10123000DF92EF92FF92CF93DF93C12CD12C7601F6
:10124000C5E0D0E0B8DE65E070E080E090E0B0D1CD
:10125000D9DE65E070E080E090E0AAD1FADE65E0DA
:1012600070E080E090E0A4D11BDF65E070E080E0FA
:1012700090E09ED1219731F7C701B60199D1C5E021
:10128000D0E0A6DE65E070E080E090E091D1C7DEBE
:1012900065E070E080E090E08BD1E8DE65E070E032
:1012A00080E090E085D109DF65E070E080E090E0CB
:1012B0007FD1219731F7C701B6017AD1C5E0D0E0DF
:1012C00094DE65E070E080E090E072D1B5DE65E02C
:1012D00070E080E090E06CD1D6DE65E070E080E008
:1012E00090E066D1F7DE65E070E080E090E060D1EC
:1012F000219731F7C701B6015BD18AE0C80ED11C36
:10130000E11CF11C84E6C816D104E104F10409F0E3
:1013100097CFDF91CF91FF90EF90DF90CF9008951E
:101320003BDE61E088E099D161E088E0E4D161E0F2
:1013300083E093D160E083E0DEC12EDE61E088E0EF
:101340008CD160E088E0D7D161E083E086D161E0B4
:1013500083E0D1C121DE61E08AE07FD160E08AE0F4
:10136000CAD161E087E079D161E087E0C4C114DED1
:1013700061E08AE072D161E08AE0BDD161E087E09E
:101380006CD160E087E0B7C107DE61E089E065D13C
:1013900060E089E0B0D161E083E05FD161E083E0AB
:1013A000AAC1FADD61E089E058D161E089E0A3D10A
:1013B00061E083E052D160E083E09DC1CF92DF9293
:1013C000EF92FF92E9DDC12CD12C7601A9DFC70194
:1013D000B601EED0B2DFC701B601EAD0BBDFC7016C
:1013E000B601E6D0C4DFC701B601E2D0CDDFC70148
:1013F000B601DED0D6DFC701B601DAD08FE0C80E65
:10140000D11CE11CF11C8BE4C816D104E104F104E9
:10141000E9F6FF90EF90DF90CF900895CF92DF92A2
:10142000EF92FF9292D0C0900401D0900501E0901D
:101430000601F0900701DC01CB018C199D09AE0972
:10144000BF09181619061A061B06ECF4B7DFA8DE4A
:10145000EEDE4DDEA1DD79D06B017C0128E833E1C1
:1014600040E050E068EE73E080E090E0BAD1C60E54
:10147000D71EE81EF91EC0920401D0920501E09229
:101480000601F0920701FF90EF90DF90CF90089552
:10149000E9ECF0E08081887F8083AAECB0E08C9159
:1014A0008C7F81608C938081877E80838081887F20
:1014B0008360808308951F920F920FB60F921124BC
:1014C0002F933F938F939F93AF93BF938091090185
:1014D00090910A01A0910B01B0910C01309108018B
:1014E00026E0230F2D3730F029E8230F0396A11DA6
:1014F000B11D03C00296A11DB11D20930801809368
:10150000090190930A01A0930B01B0930C01809103
:101510000D0190910E01A0910F01B0911001019663
:10152000A11DB11D80930D0190930E01A0930F0199
:10153000B0931001BF91AF919F918F913F912F91E7
:101540000F900FBE0F901F9018952FB7F8946091D1
:10155000090170910A0180910B0190910C012FBF3C
:1015600008953FB7F89480910D0190910E01A091DC
:101570000F01B091100122B708B600FE05C02F3F41
:1015800019F00196A11DB11D3FBFBA2FA92F982FA9
:101590008827820F911DA11DB11DBC01CD0143E023
:1015A000660F771F881F991F4A95D1F708950895F0
:1015B000CF92DF92EF92FF92CF93DF936B017C018A
:1015C000D0DFEB01C114D104E104F10479F0EFDFC5
:1015D000C8DF6C1B7D0B683E7340A0F381E0C81A26
:1015E000D108E108F108C851DC4FF2CFDF91CF916B
:1015F000FF90EF90DF90CF900895789480B783604C
:1016000080BF83B7877F83BF83B7887F836083BFB3
:1016100089B7816089BF3CDFE9ECF0E08081887F99
:10162000808380E18093670084EA809368008CEF78
:1016300080936600AAECB0E08C918C7F81608C93E3
:101640008081877E80838081887F8360808385B16D
:10165000887F866085B92F9A0895CF93DF9386FFA0
:101660000AC0982F9F73993010F48AE003C08BE072
:10167000993009F0891BE82FF0E0EC5CF04F949171
:101680008B3049F0833038F0EBE3F0E0AAE3B0E0D0
:10169000C3E6D0E006C0E8E3F0E0A7E3B0E0C2E6CE
:1016A000D0E0892F809561110DC02FB7F8949C91DF
:1016B00098239C9390819823908398818923888391
:1016C0002FBF16C03FB7623059F4F8942C91822393
:1016D0008C938081892B8083E881E92BE88307C084
:1016E000F894288182238883EC91E92BEC933FBF07
:1016F000DF91CF910895CF93DF9386FF0AC0982F93
:101700009F73993010F48AE003C08BE0993009F0A0
:10171000891BE82FF0E0EC5CF04FE4918B3059F13D
:10172000833030F0863031F480B78F7380BF28C0AB
:1017300092E001C091E0853021F480B78F7C80BFBA
:1017400018C0843019F48FB58F7304C0873021F42A
:101750008FB58F7C8FBD0DC0823021F48091CA007F
:101760008F7305C0833029F48091CA008F7C8093E9
:10177000CA00913029F0C8E3D0E0A2E6B0E004C08E
:10178000CBE3D0E0A3E6B0E08E2F80952FB76111B8
:1017900005C0F89498819823988304C0F8949881A0
:1017A000E92BE8839C9189238C932FBFDF91CF9104
:1017B0000895CF92DF92EF92FF9261157105810536
:1017C000910539F06B017C01D2D0A701960147D079
:1017D00003C060E070E0CB01FF90EF90DF90CF900E
:1017E0000895CF92DF92EF92FF920F931F936217AB
:1017F0007307840795077CF489019A016B017C01CA
:10180000C901B8016C197D098E099F09D2DF6C0DE1
:101810007D1D8E1D9F1D1F910F91FF90EF90DF90FA
:10182000CF900895EADEA8DBF9DDFECFEE27FF2793
:10183000AA27BB2708C0A20FB31FE41FF51F220F62
:10184000331F441F551F969587957795679598F395
:101850007040A9F7009799F7BD01CF010895052EB3
:1018600097FB16F400940FD057FD05D014D007FC59
:1018700002D046F408C050954095309521953F4FD1
:101880004F4F5F4F089590958095709561957F4F6C
:101890008F4F9F4F0895A1E21A2EAA1BBB1BFD017B
:1018A0000DC0AA1FBB1FEE1FFF1FA217B307E4073F
:1018B000F50720F0A21BB30BE40BF50B661F771F97
:1018C000881F991F1A9469F7609570958095909577
:1018D0009B01AC01BD01CF0108958F929F92AF9201
:1018E000BF92CF92DF92EF92FF92CF93DF93EC0102
:1018F000688179818A819B816115710581059105D6
:1019000021F464E279ED8BE597E02DE133EF41E0DE
:1019100050E0A5DF49015A0127EA31E440E050E0F8
:1019200085DF6B017C012CEE34EF4FEF5FEFC501DB
:10193000B4017CDFDC01CB018C0D9D1DAE1DBF1DF4
:10194000B7FF03C00197A109B04888839983AA8390
:10195000BB83BC01CD019F77DF91CF91FF90EF90CA
:10196000DF90CF90BF90AF909F908F9008958F920F
:101970009F92AF92BF92CF92DF92EF92FF926091CF
:1019800000017091010180910201909103016115A4
:1019900071058105910521F464E279ED8BE597E00D
:1019A0002DE133EF41E050E05ADF49015A0127EAC7
:1019B00031E440E050E03ADF6B017C012CEE34EF83
:1019C0004FEF5FEFC501B40131DFDC01CB018C0DBE
:1019D0009D1DAE1DBF1DB7FF03C00197A109B048F3
:1019E0008093000190930101A0930201B093030141
:1019F000BC01CD019F77FF90EF90DF90CF90BF901B
:101A0000AF909F908F9008956093000170930101B3
:0E1A100080930201909303010895F894FFCF94
:041A1E0001000000C3
:101D800001C021C1112484B7882371F0982F9A7063
:101D9000923051F081FF02C097EF94BF282E80E06F
:101DA000FED0EEE0FF27099485E08EBD82E08093AF
:101DB000860088E18093850086E08093840080E13E
:101DC000809381008EE0EBD0BA9A86E028E13EEF66
:101DD00091E03DBD2CBD9EB9709BFECFB29AA895F7
:101DE0004091860047FD02C0815099F7AA24A39430
:101DF00095E0992E22ECC22E2EE0D22E8D2D806CF5
:101E0000882EC1D0813461F4BED0182FCDD01238C5
:101E1000E9F0113811F488E001C083E0ADD0A9C029
:101E2000823411F484E103C0853419F485E0C4D010
:101E3000A0C0853539F4A7D0C82FA5D0D82FCC0F96
:101E4000DD1F96C0863521F484E0B6D080E0E6CF71
:101E5000843609F057C097D096D0B82E94D0782EFB
:101E600000E011E090D0F80181938F01BE12FACF0B
:101E70009BD0209769F48091000180932401809188
:101E8000010180932501C09200018092010119C0D7
:101E9000C031D105B1F4E0902401F090250180918A
:101EA0000C018093260180910D0180932701FEE0B3
:101EB000EF1AF108E0920C018F2D8F70806C8093E7
:101EC0000D0185E4781201C0FFCF8C2F8F7339F498
:101ED00083E0FE0187BFE89507B600FCFDCFFE0159
:101EE000A0E0B1E08D919D910C01A7BEE895112471
:101EF0003296BA12F7CFFE0197BEE89507B600FCFE
:101F0000FDCF37C0843739F53ED03DD0B82E3BD019
:101F10004BD08E010115110519F48091240114C0D4
:101F20000130110519F4809125010EC00C31110505
:101F300019F48091260108C00D31110519F4809122
:101F4000270102C0F801849117D0BA940F5F1F4F88
:101F5000B110E0CF0EC0853739F426D08EE10CD019
:101F600083E90AD085E15ACF813511F488E017D092
:101F70001BD080E101D045CF9091860095FFFCCF2A
:101F80008093800008958091860087FFFCCF809128
:101F9000860084FD01C0A89580918000089598ED89
:101FA0009093710081BD0895EEDF803219F088E0D2
:101FB000F6DFFFCF84E1E0CFCF93C82FE4DFC1503D
:101FC000E9F7CF91F1CFFC010A0167BFE895112431
:081FD00007B600FCFDCF0895E7
:021FFE000008D9
:0400000300001D805C
:00000001FF
